:020000040800F2
:1000000080050020D9000008191F0008591D0008AC
:1000100000000000000000000000000000000000E0
:10002000000000000000000000000000631F000846
:100030000000000000000000611F0008651F0008AC
:10004000EB000008EB000008EB000008EB000008E4
:10005000EB000008EB000008EB000008EB000008D4
:1000600000000000EB000008EB000008EB000008B7
:10007000EB000008EB00000800000000EB000008A7
:1000800000000000EB00000800000000000000007D
:10009000EB00000800000000EB000008EB00000887
:1000A000EB000008EB000008EB0000082125000829
:1000B000EB000008EB00000800000000000000005A
:1000C0000448854600F09AFB00480047852E00084A
:1000D000C046C046800500200448804704480047C9
:1000E000FEE7FEE7FEE7FEE7FEE7FEE7D91F0008B2
:1000F000C100000830B50B46014600202022012433
:1001000009E00D46D5409D4205D31D469540491B4B
:100110002546954040191546521E002DF1DC30BD94
:10012000F0B51FB40646002082B005464024019178
:1001300000901BE0019922460F46304600F086F9F8
:10014000049A059B801A994110D3104619462246FD
:1001500000F06CF9361A8F410197224601200021E8
:10016000009F00F063F938184D4100902046641E4E
:100170000028DFDC019B00982946324607B0F0BD1D
:10018000D2B201E00270401C491EFBD2704700222F
:10019000F6E710B513460A4604461946FFF7F0FF86
:1001A000204610BD024670B54A40D30FDB07400021
:1001B0002DD04A002AD0010E140E00021202091995
:1001C000400A520A8418E50104465443000A120A00
:1001D0002E045043A4194219200CC543AA18120C2E
:1001E0000125AD03521C521912047F39240400D09A
:1001F000521C104301D44000491EC2B20C06C00973
:100200002018401C4008802A02D003E0002070BD66
:1002100040084000002900DA0020184370BD420069
:1002200005D04200120E52428A4201DB0020704784
:10023000C905081870470000F0B507460846584041
:1002400087B0C00F049048000E4659004008490886
:10025000BC1A884105D2384631461E4617460B4621
:1002600002465800400810434DD0300D0390400521
:100270005900400D490D0590401A0290402873DA4C
:1002800018030121000B090508430190049800920E
:10029000002806D01146019A494200209041009161
:1002A0000190029840210A1A0199009800F0BEF8C6
:1002B00005460C466B4607CB00F0D9F8C0197141D2
:1002C000039A0E0D0023D71756401A467A4016435C
:1002D00044D0049A002A2DD0029A012A039A15DCF0
:1002E0001205C01A914101263605001C7141D20F3A
:1002F000059ED2070093019202962A46234600F0FB
:1003000017F907B0F0BD38463146FAE71605234A1B
:100310000F46B218C01AB74101210905001C4F4110
:1003200000187F41114618187941E20F10436D19EA
:10033000644113E0E2076D0815436408C2071443E3
:10034000039A01261205C01A91413605001C71411D
:10035000CE07400830434908C01851412A46234679
:1003600000F0D9F8CDE7FFE7049801224000C1175B
:10037000121A00238B4104983146C417381AA14140
:10038000EEE730B40124E407634030BC54E730B4F6
:100390000124E407614030BC4EE700000000E0FFAC
:1003A00010B500229623114600F07CF810BD000025
:1003B0000EB505490291002100910A460B460191B4
:1003C00000F0B6F803B000BD33040000C20FD2073E
:1003D000400040080BD0C10D0723DB01C9184002C3
:1003E0000905400A1143C208400711437047002025
:1003F00001467047CB0FDB07490010B5490802469C
:100400000A4307D00A0D07240903E401090B121B54
:10041000002A01DC002010BDC900440F0C43C100BC
:10042000E018D205801800F035F810BD10B5202A6C
:1004300004DB0146203A9140002010BD914020236A
:100440009C1A0346E3401943904010BD10B5202A82
:1004500004DB0846203AD040002110BD0B46D340B3
:10046000D0402024A21A91400843194610BD10B56F
:10047000202A06DBCB170846203A1041C1170B4350
:1004800006E00B461341D0402024A21A91400843B5
:10049000194610BD002904DA401C490001D140086A
:1004A0004000704770B40024050C05D110240004EE
:1004B00002D1002921D01124050E01D100020834F7
:1004C000050F01D10001241D850F01D18000A41C5E
:1004D000002801DB4000641C002908D020252E1BC9
:1004E0000D46F540A14000D00121294308430106F3
:1004F0001B1B000ADB1D02D5002070BC7047DB050A
:10050000181880180029F8DA401C4900F5D170BC91
:1005100040084000704710B5002B08DA0024401C4A
:10052000614192185B411A4301D14008400010BD5F
:10053000F0B51FB482B005460C0003D0084602F0A7
:1005400007F802E002F004F820300246009021464D
:100550002846FFF76BFF049B059A04460F46184395
:100560001143084314D0184610431BD00098402173
:100570000A1A18460599FFF769FF05460E46009AC4
:1005800005990498FFF752FF084305D0012004E0C5
:100590002046394607B0F0BD0020C11705430E4381
:1005A0002C43374300990E986305401A7905E40AF5
:1005B00000220C43FD0A0A3002D500200146E9E77B
:1005C0000105101969410C9C0D9D00196941FFF747
:1005D000A2FFDFE7F0B51FB488B00B99099800249B
:1005E00048400999C00F490049080991C0070B9973
:1005F0000090490049080B9109990898A6460843BC
:100600001CD00B990A98084318D00998012440007F
:10061000420D4800410D099824050003000B2043BA
:1006200009900B980003000B20430B9050181C49B5
:100630004018002201901446104605E000200146B3
:100640000DB0F0BD032801DA034600E003239C4609
:10065000C11A0AAE0AE05F0008ADED5B4F00F75B20
:100660007D430027AA187C41491C5B1E6145F2DDD1
:10067000410004AB5A522104120C0A43240C401CC2
:100680000828DFDB019802900099704601910090E4
:10069000059B049A07990698FFF74AFFD0E70000E8
:1006A0000DFCFFFFF0B50C465C4085B0E40FE4079D
:1006B00003944C00002664085900944649080246F9
:1006C0000296224321D062460A431ED06200570D93
:1006D0004A000E032303550D012402462C4924052C
:1006E000781B1B0B360B40182343264361460090B2
:1006F0001C46501AB44103D30098401C009002E0FD
:10070000921800985B41002803DA0020014605B0EA
:10071000F0BD0020012109050746864611E0644628
:100720001D46141BB54106D36546521BB3417446A2
:1007300007430C43A646CD074008490828439218B2
:100740005B4105460D43EAD11046184313D060467D
:10075000194650407140084306D06046101AB34114
:1007600006D20122002306E000220123DB0702E07B
:100770000122D2435310009874460105381C614190
:10078000029C039D00196941FFF7C5FEBFE7000009
:10079000FD0300004A0009030123090B1B0519434F
:1007A0000A4B10B5520D9A4202DA0020014610BDE4
:1007B000064B34339A4203DC9A1AFFF747FE10BD0A
:1007C000034BD218FFF732FE10BD0000FF030000FC
:1007D000CDFBFFFF10B5002904DB0124E4074042F4
:1007E0008C412146002B04DB1C460123DB075242CF
:1007F000A341994200D1904210BD0000064C012552
:10080000064E05E0E36807CC2B430C3C98471034B8
:10081000B442F7D3FFF758FCA02F0008C02F000800
:1008200038B50446064805490068FFF763FC604395
:1008300000E0401E00900028FBD138BD40420F0070
:1008400010000020F8B50446006881688907890F08
:10085000012902D10168C90722D18168114A1026F5
:100860001140012500290ED18168294381600120B2
:10087000FFF7D6FF00F0FAFA07460CE000F0F6FAB0
:10088000C01B0A2807D9606D30436065A06D2843FE
:10089000A0650120F8BD20680068C043C007EDD105
:1008A0000020F8BD1700008070470000F8B506462C
:1008B0000D464036317C01290DD00121317401688B
:1008C0008A68520709D5416D2022114341650020F5
:1008D00030740120F8BD0220F8BD174B6A68D805B6
:1008E00047109A42154C8A6A2B6812D05B035B0B47
:1008F0001A438A622968490305D5A1680143A160AA
:100900000A20FFF78DFF2868800312D5A0683843BE
:100910000EE05B035B0B9A438A622968490302D5A8
:10092000A1688143A1602868800302D5A068B8430C
:10093000A06000203074F8BD0110000000270140C5
:10094000406D70470068006C7047000070B504008F
:1009500006D0606D264600254036002802D006E00D
:10096000012070BDA5653574204600F0D3F8606D98
:10097000C00603D421688868400705D5606D102142
:10098000084360653574EBE7606DFF2201329043E8
:1009900002221043606588688207920F5B48012A33
:1009A00002D10A68D2072BD1032362689B079A42BF
:1009B00005D05B429A4202D05B009A4209D10A6993
:1009C000920092080A6121680A6963681A430A6101
:1009D0000CE00A69920092080A6181680F22920471
:1009E0009143816081686268114381602168CA68AF
:1009F00018239A43CA602168CA68A3681A43CA6068
:100A0000816801225206914381608168A28E52065C
:100A10001143816020688168C90004D48168012283
:100A20001207114381602068C168394A1140C160D2
:100A30002069E168022825D00020014320462030AB
:100A40000278037B52035B001A431143226B11436C
:100A5000A26992031143E269D20311432268D36869
:100A60001943D160616A0A46FF3AC23A05D0A26AC8
:100A700011432268D3681943D16042780121012AC9
:100A800002D00BE00420D8E70078002823D0606D66
:100A9000202210436065A06D0843A065E06B01282B
:100AA00020681FD00169C90703D0016949084900BE
:100AB000016120684169C908C90041612068416934
:100AC000A26B11434161A565606D80088000401CE8
:100AD0006065002070BD2068C26801231B041A43B2
:100AE000C260DBE70269FF239B009A430261206832
:100AF0000269236CA66C1A43636C33431A43026188
:100B0000206802690A430261D3E700000027014020
:100B10001902FEFF10B586B0044614216846FFF79F
:100B200036FB0E492068884216D10D48416B4215AC
:100B300011434163C16A01221143C162C06A69461F
:100B4000104005901020009003200190002002909A
:100B50000520000700F0C8F806B010BD00240140D1
:100B600000100240F8B504464069254640350E465F
:100B700008280BD02068C068C00709D0606D20210C
:100B800008436065002028740120F8BD082700E0B4
:100B90000C2700F06BF9009011E0701C0FD0002EB4
:100BA00005D000F063F90099401AB04207D9606D92
:100BB000042108436065002028740320F8BD2068E4
:100BC00000683842E9D0606D012149020843606540
:100BD0002068C16809058A0F0C21002A1BD1202238
:100BE000125D002A17D10268120714D582685307D4
:100BF0000122002B08DB43688B434360606D1302C6
:100C000098431043606506E0606D202318436065DB
:100C1000A06D1043A065A069002801D12068016083
:100C20000020F8BD70B50446216800208968490796
:100C300021D425464035297C01291CD00121297465
:100C4000E169012904D02046FFF7FCFD002811D1FD
:100C5000616D0A4A1140FF22013211436165002192
:100C6000A165297422681C21116021688A68042307
:100C70001A438A6070BD022070BD0000FEF1FFFFC4
:100C800070B50024014620314A79022A03D004219C
:100C9000C163012418E0026813680E25AB4313609A
:100CA000026813685B085B001360436C1C221340EE
:100CB000012215469D40036C5D604A7100220A7155
:100CC000816B002900D08847204670BD70B504466E
:100CD00000F0CCF80546601C00D0641C00F0C6F89B
:100CE000401BA042FAD370BDF8B500230124A2E056
:100CF00027469F403A4070D04D68022D01D0122DFA
:100D000014D1DD08AD002D1800952D6A5E07AC46A4
:100D1000F50E0F26AE46AE406546B543AC460E69AD
:100D20007546AE4065462E43009D2E624D68012DEE
:100D300005D0022D03D0112D01D0122D16D18568BA
:100D40000326AC465D00AE46AE406546B543AC46B4
:100D5000CE687546AE4065462E43866046680D797E
:100D6000BE43ED06ED0F9D403543456006685F00CC
:100D70000325BD40AE46AE430D79B446AE07B60F6F
:100D8000BE4065462E430660C6687546AE438D6814
:100D9000BD403543C5604D68ED004BD5294D6E6BA8
:100DA00026436E639E08284DB6007519AC46AD68A3
:100DB0009E07360F0F27B740BD4305273F07B842B0
:100DC00001D1002715E0214FB84201D1012710E0E1
:100DD0001F4FB84202D102270BE02BE01D4FB84253
:100DE00001D1032705E01C4FB84201D1052700E0DF
:100DF0000627B7402F436546AF60184D2E684F68F1
:100E00009643FF0300D516432E606E684F689643E5
:100E1000BF0300D516436E60AE684F689643FF026D
:100E200000D51643AE60EE684F689643BF0200D50A
:100E30001643EE605B1C0A681546DD4000D057E79C
:100E4000F8BD000000100240000001400004005006
:100E500000080050000C0050001C0050000401402D
:100E6000002A01D0816170478162704701480068A3
:100E7000704700000C00002070B5024640325378E5
:100E8000202B1CD11378012B19D00123137024249B
:100E90005470046825689D432560046825681E0316
:100EA000B5432560046825680D4325600068016826
:100EB00019430160202050700020107070BD022086
:100EC00070BD70B5024640325378202B1BD1137889
:100ED000012B18D0012414702423537003681D685B
:100EE000A5431D6005682B680F263602B34309022F
:100EF0001943296000680168214301602020507077
:100F00000020107070BD022070BD000070B504009C
:100F100006D02546403568780026002802D005E036
:100F2000012070BD2E70204600F04AF82420687021
:100F3000206801684908490001600F2160680906BE
:100F400088432168086121688A680120C0038243C0
:100F50008A60E1680129A16808D021229202114328
:100F600022689160E168022902D005E00143F7E7B9
:100F700001212268C902516021684A680F4B1A4357
:100F80004A602168CA688243CA606169206908436F
:100F9000A169090208432168C860216AE069084321
:100FA00021680860206801680122114301606664BD
:100FB000202068702663AE70002070BD00800002A3
:100FC00010B586B0044614216846FFF7E0F81149D1
:100FD000206888421BD1104CE16A02200143E16283
:100FE000E16A0140032005918002009012200190E7
:100FF00001200290032003900620049069460748D0
:10100000FFF772FEA06B012189050843A06306B0BB
:1010100010BD0000005800400010024000040050C5
:1010200002480168491C0160704700000C00002064
:1010300010B5084800240168402211430160204691
:1010400000F00AF8002801D0012401E000F01CF8AB
:10105000204610BD0020024070B5054609487D219C
:101060000024C9000068FFF745F800F0F9FB0028EC
:1010700001D0012404E000222946501E00F01AF895
:10108000204670BD100000200448416B012211432E
:101090004163816B02041143816370470010024079
:1010A000C106C90E01208840014908607047000050
:1010B00000E100E010B500F031FF10BDF8B50446C6
:1010C0000078544D800672D5524E0027403EB06BDA
:1010D000C00004D4B06BA9050843B06301274E4893
:1010E0000168C90511D40168821511430160FFF739
:1010F000BDFE009005E0FFF7B9FE0099401A642894
:1011000037D845480068C005F5D532680321090580
:1011100060680A400140914208D08103890F032989
:1011200004D13168890301D50120F8BD2A69032162
:1011300009040A4022D0084090421FD0207880063F
:101140001CD528692A6988430121C9040A432A61F8
:101150002A698A432A612861C0050FD5FFF786FEF8
:10116000009008E0FFF782FE0099411A2B48814267
:1011700001D90320F8BD28698005F3D5616888038B
:10118000800F032805D132680005824301400A43DD
:101190003260286903226168120411400843286103
:1011A000002F04D0B16B012000078143B163207888
:1011B000C00705D0E868A168800880000843E8609F
:1011C0002078800705D5E8680C218843E16808434A
:1011D000E8602078400706D5E86803218902884343
:1011E00021690843E8602078000706D5E8680321F4
:1011F0000903884361690843E8602078000606D542
:10120000E868032189048843A1690843E860002055
:10121000F8BD00004010024000700040881300003C
:10122000F8B50E4605007DD053480068C007C00FD2
:10123000B0420AD250480168490849003143016070
:101240000068C007C00FB04271D128784B4C8007AE
:1012500005D5E068F0218843A9680843E060287854
:10126000C00752D06868022817D0032818D0216818
:10127000012818D08905002959DAE1688908890010
:101280000143E160FFF7F2FD69680746022912D0C9
:1012900003291CD0012926D033E021688903EAE71D
:1012A00021688901E7E74907E5E7FFF7DFFDC11B93
:1012B0003348814223D8E0680007800F0228F4D128
:1012C00023E0FFF7D3FDC11B2D48814217D8E0680A
:1012D0000007800F0328F4D117E0FFF7C7FDC11BFB
:1012E000274881420BD8E0680007800F0128F4D11D
:1012F0000BE0FFF7BBFDC11B2148814201D9032050
:10130000F8BDE0680007800FF3D11B480168C907EA
:10131000C90FB1420DD90168490849003143016044
:10132000006800E003E0C007C00FB04201D0012018
:10133000F8BD2878400706D5E068072109028843F0
:10134000E9680843E0602878000707D5E0680721CE
:10135000C90288432969C9000843E06000F036F8F3
:10136000E168084A0906090F515CC840064908604F
:101370000020FFF771FEF8BD00200240001002407F
:10138000881300007C2F0008100000200448054945
:101390000068C968044A4905490F515CC840704754
:1013A0001000002000100240952F00080448054955
:1013B0000068C968044A8904490F515CC8407047F5
:1013C0001000002000100240952F000810B5184AA8
:1013D000D1680C20084004280BD0082810D00C2815
:1013E00010D050680004410F0120C003491C884000
:1013F00010BD1068C00601D50E4810BD0E4810BDC6
:101400000E4810BD88020E4B000F185C0902D3680D
:10141000890F491CDB0301D5084A05E01268D20692
:1014200001D5044A00E0044A5043FEF763FE10BDB4
:101430000010024000093D000024F40000127A0070
:101440008C2F0008FEB505007ED0FE4CE7680C200E
:10145000E66807400120000406402878C00747D00E
:10146000082F05D00C2F0AD101200004864206D196
:10147000206880033CD568680028E5D038E001206A
:1014800069680004814203D121680143216011E0B1
:10149000052301221B0492049942216802D11143C1
:1014A0002160F1E7814321602168014000912068BB
:1014B00090432060686800280DD0FFF7D7FC0090AB
:1014C00005E0FFF7D3FC0099401A64287AD8206819
:1014D0008003F6D50CE0FFF7C9FC009005E0FFF7AC
:1014E000C5FC0099401A6428F0D820688003F6D41F
:1014F0002878800755D50923E868042F0DD00C2FD4
:1015000001D1002E09D000283BD021689943014326
:101510002160FFF7ABFC064627E02168490701D5AB
:10152000002891D061681F22120291432A69120299
:10153000114361602168994301432160FFF746FF31
:10154000E16809060A0F00E079E1BF49895CC840FB
:10155000BE4908600020FFF77FFD002872D120E01F
:10156000FFF784FC801B0228B0D820684007F7D51D
:1015700060681F21090288432969090208436060E5
:101580000FE02068400840002060FFF76FFC06462F
:1015900004E0FFF76BFC801B022897D82068400707
:1015A000F7D42878C0065FD5002F0CD0A869002892
:1015B00049D02068FF21013108432060FFF756FC25
:1015C00006462DE0C0E02068800502D5A869002805
:1015D000A7D06068072149038843296A08436060EF
:1015E0006068297F0002000A090608436060286AD3
:1015F000410B0120C003491C8840E16809060A0F1D
:101600009149895CC840914908600020FFF724FD9A
:10161000002817D128E0FFF729FC801B0228A3D857
:1016200020688005F7D56068072149038843296A47
:10163000084360606068297F0002000A09060843C9
:10164000606011E0E1E02168FF200130814321600A
:10165000FFF70CFC064604E0FFF708FC801B02289D
:1016600072D820688005F7D42878794E000724D5F1
:1016700068690028306910D0012108433061FFF704
:10168000F5FB009005E0FFF7F1FB0099401A0228F6
:101690005AD830698007F6D50FE040084000306125
:1016A000FFF7E4FB009005E0FFF7E0FB0099401A2C
:1016B000022849D830698007F6D42878400765D5D4
:1016C00000200290A06BC00006D4A06B0121090786
:1016D0000843A063012002905E480168C90511D447
:1016E0000168821511430160FFF7C0FB009005E01F
:1016F000FFF7BCFB0099401A642825D855480068BC
:10170000C005F5D5FF20AA680130824203D13169B6
:101710000143316111E001218902002A07D005232C
:101720001B029A4203D132690A433261EFE7326900
:1017300082433261306988433061A86800280FD045
:10174000FFF794FB009007E05EE0FFF78FFB009946
:10175000411A4148814257D830698005F5D50DE0DE
:10176000FFF784FB009006E0FFF780FB0099411A29
:101770003948814248D830698005F5D4029800285C
:1017800004D0A06B012109078843A063686A002880
:1017900064D00C2F3ED0012636060228206805D0E2
:1017A000B0432060FFF762FB05462FE0B0432060A6
:1017B000FFF75CFB074604E0FFF758FBC01B02285D
:1017C00022D820688001F7D4E96AA86AE268084351
:1017D000296BFD231B049A4311430843E0602068F2
:1017E00030432060FFF742FB054604E0FFF73EFB75
:1017F000401B022808D820688001F7D52EE0FFF7AB
:1018000035FB401B022801D90320FEBD2068800162
:10181000F5D423E00128F8D0E06801210904AA6A80
:10182000014091420BD10F218904EA6A01409142A3
:1018300005D1032189050840296B88420ED001207B
:10184000FEBD0000001002407C2F000810000020A8
:101850004010024000700040881300000020EFE7B5
:10186000094910B5401E884201D9012010BD074C1E
:1018700060610321081F00F051FB0020A0610720D8
:101880002061002010BD0000FFFFFF0000E000E02D
:10189000F0B502462032137E012B15D001271776B2
:1018A0000223537605686C68AB687026B4430E68F3
:1018B000496826438024A34319436E600068816011
:1018C000577600201076F0BD0220F0BD70B5040000
:1018D00005D025462035687E002802D006E001208C
:1018E00070BD00202876204600F00AF802206876B5
:1018F000211D206800F09AFB01206876002070BD51
:1019000000680449884204D10348816B10221143C6
:10191000816370470010004000100240704770471C
:10192000F8B502680446D0691168936805072D0F61
:101930005BD0DD07ED0FFF2621360E402E4367D02A
:10194000C60706D0CE0504D501261662E26F3243E3
:10195000E267870702220426002F06DADF0704D099
:1019600027683A62E76F3743E767470706D5DB0723
:1019700004D023681E62E36F1343E367020709D5AF
:1019800020220A402A4305D0236808221A62E36F06
:101990001343E367E26F002A2FD0800606D588063E
:1019A00004D5216E002901D020468847E06F2168C8
:1019B0008968490601D4000724D5204600F002FCBE
:1019C00020688168490619D5816840229143816069
:1019D000E06E002812D020498163E06EFFF750F9D5
:1019E00000280AD0E06E816B06E0850610D58D06D2
:1019F0000ED5216E1CE020468847F8BD2046FFF733
:101A00008EFFF8BD2046FFF78AFF0020E067F8BD93
:101A1000C50208D55B0206D50120000510622046EC
:101A2000FFF77CFFF8BD030605D50B0603D5616EF5
:101A30000029E0D1F8BD4006FCD54806FAD5136868
:101A4000204640218B43136020216167002161669D
:101A500000F081F9F8BD0000B121000810B50400C4
:101A600003D0606F002802D007E0012010BD0021E4
:101A700070200155204600F027F824206067206878
:101A80000168490849000160204600F003FC012874
:101A9000ECD0606A002802D0204600F0F3FA2068FB
:101AA00041680922D20291434160206881682A225C
:101AB0009143816020680168012211430160204642
:101AC00000F046FB10BD000010B586B0044614219E
:101AD0006846FEF75CFB15492068884224D114480B
:101AE000416B0122920311434163C16A01221143F8
:101AF000C162C06A69461040059003204002009010
:101B00000220019000200290032003900420049002
:101B100005200007FFF7E8F8002211461B20FFF719
:101B2000C9FA1B20FFF7BCFA06B010BD003801400F
:101B300000100240F0B5836F202B54D100290AD049
:101B4000002A08D08568DC01A54206D10369002B74
:101B500003D1CB0701D00120F0BD034660331E7CCA
:101B6000012E40D001261E744165014640310A8392
:101B70004A830022FF260266A54204D10569002D92
:101B800013D11A4D0AE07F27002D09D00126360710
:101B9000B5420CD10569002D05D03F258D8307E0A6
:101BA0000569002D01D08F8302E08E8300E08A83D7
:101BB000C2672221816701688D68012635438D60E7
:101BC0008168A14202D1016900290AD00849016651
:101BD0001A7400680168FF2221321143016000205D
:101BE000F0BD0449F3E70220F0BD0000FF01000052
:101BF0003D220008E5210008F8B500681D4988422B
:101C000036D11D4C2078002832D16078A61E0028DD
:101C10002DD001282CD11948FFF704F8322117489C
:101C2000FEF7A0FF1548FEF78BFE800520D5134870
:101C3000FEF788FE87B23780A078FEF7B9FB002256
:101C40000F4BFEF7F9FA04460D463846FEF7A8FB9F
:101C50000C49FEF7A7FA0B21C943FEF7E0FAFEF79D
:101C6000B5FB22462B46FEF78CFBFEF7C3FBB060AC
:101C7000F8BD0000003801400200002018000020DC
:101C80000000F83F33335340FFB50446406F83B044
:101C900017460D4620285CD1002D0AD0002F08D011
:101CA000A168C001814207D12069002804D1E8075A
:101CB00002D0012007B0F0BD204660300290007CC9
:101CC000012846D00298012101740020E0672120FC
:101CD0006067FFF7CBF8264640360190378277825F
:101CE0000120A1680003814202D12069002802D0AE
:101CF0002F46002511E000270FE00022802120461A
:101D000000F0DCFB002815D1002F15D021683878B1
:101D100088627F1C708A401E7082708A019B002836
:101D200006980090E9D100224021204600F0C6FB31
:101D3000002808D00320BDE728882168C005C00D11
:101D40008862AD1CE6E720206067029900200874D5
:101D5000B0E70220AEE77047FEE700001CB50021A7
:101D600018480091164A01910260C1631205426051
:101D700081600122826302610246C16020321170DB
:101D8000FF235170C2334362816211730163816129
:101D9000042241634261C161FEF7D8FD002801D0F1
:101DA000FEF782FD0848009000140190694605483E
:101DB000FEF77CFD002801D0FEF776FD1CBD00007B
:101DC000002401401800002010000010F0B587B07A
:101DD00014216846FEF7DBF91848C16A012529433A
:101DE000C162C16A29400591C26A02210A43C262E6
:101DF000C06A032408400526E40236070590002245
:101E000021463046FFF72CF80D4F0022702138464E
:101E1000FFF726F8009400240195029469463046A5
:101E20000394FEF761FF70200090029469460195CB
:101E300003943846FEF758FF07B0F0BD001002408B
:101E40000004005010B5144812490160E121C90096
:101E50004160002181600161416181610122C161B4
:101E6000C2600162FFF752F8002801D0FEF71CFDA6
:101E700000210948FFF700F8002801D0FEF714FD03
:101E800000210548FFF71DF8002801D0FEF70CFDE2
:101E900010BD000000580040740000201CB5002454
:101EA0000E4800940C490194016007218460416050
:101EB00001214461C160FFF709FD002801D0FEF750
:101EC000F3FC0094694605480194FFF7E1FC002803
:101ED00001D0FEF7E9FC1CBD00100040C00000204E
:101EE00010B50C480A490160E12149024160002116
:101EF0008160C16001618161C1610C220162426146
:101F00004162FFF7ABFD002801D0FEF7CDFC10BD0C
:101F100000380140FC000020704700008307FF22CA
:101F2000DB0E9A408907090E994000280BDA00075A
:101F3000000F0838830808489B001818C3699343AA
:101F40000B43C3617047830804489B001B18186843
:101F5000904308431860704700ED00E000E400E0A3
:101F60007047704710B5FFF75BF810BD30B599B0FA
:101F700034216846FEF70BF914210DA8FEF707F986
:101F80001C2112A8FEF703F9124801680322D202AD
:101F90009143C2148918016002200090002410208F
:101FA00009940125049003956846FFF74BFA0F202A
:101FB0000D9080200F900E951094002111940DA883
:101FC000FFF72EF912A812951494FFF777F819B0BD
:101FD00030BD0000007000401048016882151143B8
:101FE0000160C1680E4A1140C16001680D4A11408C
:101FF00001608168490849008160016801229204FA
:1020000091430160C168FD2212049143C160002127
:1020100001610549C003886070470000001002405C
:102020000C40FF88F6FFF6FE00ED00E070B5026898
:1020300001239B07114C124D984203D0A04201D0BE
:10204000A84203D17026B2434E683243984203D06F
:10205000A04201D0A84204D103231B029A43CB68BB
:102060001A4380239A430B691A4302608A68C2624A
:10207000096881620121416170BD000000080140D2
:102080000014014010B5818CC90707D001684A6867
:1020900001235B049A43836A1A434A60818C89074F
:1020A00007D501684A6801231B049A43C36A1A438F
:1020B0004A60818C490707D501684A6801239B045F
:1020C0009A43036B1A434A60818C090707D501685C
:1020D0004A680123DB039A43436B1A434A60818CAD
:1020E000C90607D50268916801231B039943836BD6
:1020F00019439160818C890607D501688A6801239C
:102100005B039A43C36B1A438A60818C490612D5DC
:1021100003685A6801210905046C8A4322435A6006
:10212000026C8A4207D10268516803235B05994318
:10213000436C19435160818C090607D501684A68D0
:102140000123DB04806C9A4302434A6010BD000007
:10215000F8B500260446C667FEF788FE05462068E7
:102160000068124F000709D501212B4600224905BE
:102170002046009700F0A2F900280DD120680068E1
:1021800040070BD501212B460022890520460097E8
:1021900000F094F9002801D00320F8BD20206067EA
:1021A000A067603426740020F8BD0000FFFFFF0127
:1021B00010B5806A0022014640314A834A82FFF707
:1021C000AEFB10BD01680A68FF2321339A430A6001
:1021D00001688A68520852008A60202181670021C4
:1021E0000166704710B5014640318B8B846F0268E1
:1021F000222C04D0906908210843906110BD526AD6
:10220000446D1A402280426D921C42654A8B521ED8
:102210004A83498B0029F1D101680A68FF232133E1
:102220009A430A6001688A68520852008A60202135
:10223000816700210166FFF7DFFC10BD10B5014684
:1022400040318B8B846F0268222C04D09069082166
:102250000843906110BD526A1A40436D1A70426D76
:10226000521C42654A8B521E4A83498B0029F1D188
:1022700001680A68FF2321339A430A6001688A686B
:10228000520852008A602021816700210166FFF711
:10229000B3FC10BDF8B504462669A268E76932436D
:1022A0006669102000253E432368324378491E6842
:1022B000784F3E4016431E6023685A680326360353
:1022C000B243E66832435A602368A2698B4201D068
:1022D000266A32439E680B273F02BE4316439E6028
:1022E0006D4E23686D4AB3420CD1D2689207920FAB
:1022F00006D0012A38D0022A34D0032A20D11EE089
:1023000001201DE0664EB3420AD1D2680C2632404D
:1023100026D0042A28D0082A24D00C2A10D10EE076
:102320008B420DD1D66803229202164018D00122AA
:102330009202B61A18D0B61A14D0964200D10820CC
:10234000564A0126403A574FF6038B4236D10028B1
:102350000CD002280DD0042812D008281FD11CE070
:102360000020EDE70220EBE70420E9E7FFF70EF895
:1023700008E01068C00601D5384605E04A4803E089
:10238000FFF724F8002873D0626851005118814289
:1023900005D81103814202D303E03046F4E701255A
:1023A00066E0010E06025008002330185941FDF77F
:1023B000B7FE03210902411A3C4A55E0E169B142E6
:1023C00032D1030000F0DBF809070A0D06250606E6
:1023D000062B0600E3E7FEF7D9FF1CE0FEF7E6FF59
:1023E00019E010686168C00602D54808304A01E06B
:1023F000304A48088018FDF77DFE80B201462E4A1B
:1024000010399142CBD8511C01400007400F0843BE
:102410002CE0FEF7DBFF616840004A08EAE76168EC
:10242000012248081204E5E7030000F0A8F80907B4
:102430000A0D06260606062C0600B0E7FEF7A6FFE4
:102440001DE0FEF7B3FF1AE010686168C00602D510
:102450004808C01902E014484A081018FDF74AFE5F
:1024600080B20146144A1039914298D82168C86058
:102470000020206660662846F8BDFEF7A7FF616869
:102480004A088018EAE7616848088019E6E7000012
:1024900000480040F369FFEF00380140401002405F
:1024A0000044004000093D000024F400FFFC0F0040
:1024B00000127A000048E801EFFF0000FFB581B08C
:1024C00017460E4604460A9D09E0681C07D0FEF731
:1024D000CDFC0499401AA8420CD8002D0AD02068DF
:1024E000C1693046884318D00020B842EDD00020A2
:1024F00005B0F0BD20680168FF22A1329143016060
:102500002068816849084900816020206067A067D1
:102510000020603420740320EAE70120E5E7000092
:1025200010B50248FFF7FCF910BD0000FC000020C8
:102530000FB410B503A9044B044A029800F0F6F852
:1025400010BC08BC04B01847692E00081400002015
:102550002021020C01D010211046020A01D01046A1
:102560000839020901D01046091F820801D010461F
:10257000891E420801D0881E7047081A704730B47F
:102580007446641E2578641CAB4200D21D46635D10
:102590005B00E31830BC184702E008C8121F08C1EE
:1025A000002AFAD170477047002001E001C1121FD4
:1025B000002AFBD170470000F0B51FB486B009981F
:1025C000089A030D0021024314D05148514A1818AB
:1025D000504305141198012810981AD0281A401C4D
:1025E00000264D4F4D49009601910490002812DAC3
:1025F000444211E01198012449A3012801D1109807
:10260000C1430698119A84600360C26041600BB0B8
:10261000F0BD4042E4E70446210500203F4A001C8B
:1026200051410391029012E0E00707D032463B4649
:1026300001990098FDF7CEFF0191009032463B468C
:1026400010461946FDF7C6FF06460F466410002CDB
:10265000EAD10498039B0028029A0999089806DA9F
:10266000FDF7B8FF019B009AFDF7B4FF05E0FEF708
:1026700019F8019B009AFEF715F804460E46002251
:10268000284BFEF7A7F803D80020C043014607E017
:102690000022254B20463146FDF7CEFDFEF77AF8A5
:1026A000102409E0002C0ADB0A220023FDF738FD84
:1026B000079B30321A55641E02460A43F2D111229A
:1026C000641C079B121B1C19119B012B03D00123B7
:1026D00008430ED10AE0084304D0112010900020D6
:1026E000119077E71098151A6D1E0BE01098824232
:1026F00002DD00236D1C03E0824201DA00236D1E1F
:10270000002BEED0069811998260C16030C07EE740
:1027100001FCFFFF104D0000000014400000F03FDE
:10272000300000000000F0430000E03FFFB597B02C
:10273000064600251BE2252876D100242746F749C6
:10274000049400E00443761C32780120203A904043
:102750000842F7D130782A280ED00222307801467C
:102760003039092916D804990A23594330394018B9
:102770001443761C0490F1E7189802C8049118904D
:10278000002904DA01204003044348420490022057
:102790000443761C30782E2814D10420044370782A
:1027A000761C2A2809D11898761C80C8189009E050
:1027B0000A214F43303FC719761C30780146303923
:1027C0000929F5D930786C2810D006DC4C281AD0AD
:1027D00068280ED06A2817D104E0742813D07A280C
:1027E00012D110E00120400504430CE0012109054D
:1027F00001E0032109050C437178814203D10120D6
:1028000000052418761C761C307866280BD013DC63
:1028100058287DD009DC00287BD04528F6D04628F2
:10282000F4D047281AD1A9E118E0632835D06428EC
:1028300070D0652812D1A1E170286CD008DC67281F
:10284000F1D069287DD06E280DD06F2806D1BCE06C
:1028500073282ED0752873D0782859D01A9A1999D0
:1028600090476D1C82E16002400F022809D00328C6
:102870000DD00428189801680DD00D60001D189027
:1028800074E11898EA1701680D604A60F6E7189835
:1028900001680D80F2E70D70F0E718986A4601783C
:1028A0001172001D18900020507202A800900120A3
:1028B00005E0189802C8189000200091C0436107F5
:1028C0000ED5002101E00199491C0191B94213DAAA
:1028D0008142F8DB019A0099895C0029F3D10BE071
:1028E000002101E00199491C01918142FADB019A22
:1028F0000099895C0029F5D1019904981A9B471A1F
:1029000021463846199A00F099FA4019019903E0D6
:1029100051E030E115E050E0451807E000980099DB
:102920000078491C00911A9A199990470198401E05
:102930000190401CF2D1214638461A9B199A12E1A7
:1029400037E00A200021009001916002410F022926
:1029500007D0189A01CA1892C2179446032908D0C2
:102960000AE01898C01DC108C90005C9189194460D
:1029700007E000B2C2179446042902D140B2C11741
:102980008C4600226146944506DA0A460021404200
:1029900091418C462D2102E0210504D52B216A4668
:1029A0001173012103E0E10701D02021F7E7029133
:1029B00056E00A200AE0102008E0102000900021D4
:1029C000042004430191082703E00820002101911D
:1029D00000906002410F022907D0189A01CA18928C
:1029E00000229446032908D008E01898C01DC108A9
:1029F000C90005C91891944603E080B2042900D1AA
:102A0000C0B20021029121072AD531780D91702999
:102A100006D0009A1021019B4A401A4305D00EE0CF
:102A200040216A461173012108E06146014306D046
:102A300030216A4611730D99517302210291009A57
:102A40000821019B4A401A430AD16146014301D142
:102A5000610705D530216A46117301217F1E02915D
:102A60003178582904D02EA10E910DA90D910DE0B9
:102A700030A1F9E76146019B009AFDF751FB0E9BDF
:102A80008C469B5C0D9A521E0D9213706146014359
:102A9000F0D10D9805A9081A20300190600703D5E0
:102AA00001200004844300E001270198874201DDF2
:102AB000381A00E000200199009041180298091886
:102AC0000498401A0490E00306D421461A9B199AF0
:102AD000049800F0B3F94519002706E003A81A9AF4
:102AE000C05D199990476D1C7F1C02988742F5DBE9
:102AF000E0030CD521461A9B199A049800F09EF920
:102B0000451904E01A9A3020199990476D1C0099D4
:102B1000481E00900029F5DC1FE000000928010094
:102B20003031323334353637383961626364656643
:102B30000000000030313233343536373839414205
:102B400043444546000000000D980D990078491C4B
:102B50000D911A9A199990476D1C0199481E019080
:102B60000029F1DC4DE100F059F94519761C307867
:102B7000002800D0DFE528461BB0F0BD600700D478
:102B800006271898C01DC108C90048680A6808319E
:102B9000C30FDB071891190001D09CA108E02105A3
:102BA00001D59BA104E0E10701D09AA100E09AA120
:102BB0004300109130785B0865280CD006DC45286E
:102BC00009D046281DD0472841D141E0662818D0B9
:102BD00067283CD13CE00021112F01DB112000E0EF
:102BE000781C0191009008A911A8FFF7E5FC139942
:102BF00005910021119A15927F1C1298019700915E
:102C000050E00120C00703900120019008A900971F
:102C100011A8FFF7D1FC139A149905920022119B79
:102C2000009212981593059A0192002901D010463E
:102C300002E0791C40180190381A01D5019804E08F
:102C40004042401E0090781C0190C01B029043E05F
:102C5000012F00DA01270021112F01DD112000E0F2
:102C600038460191009008A911A8FFF7A5FC139917
:102C70000591119A00211298159200910197210750
:102C80000CD40599B94201DB019900E001910129B9
:102C900004DD159A491E515C302906D0B84201DA8C
:102CA000011D05DA0121029115E00199491EEDE7A8
:102CB000002805DC0099411800910199091A03E0E8
:102CC000019A411C914200DD01910099401A401C7B
:102CD00002900120C0070390200706D402990198B2
:102CE000814202DB0020C043029000206946C87781
:102CF00007AF012103980337C907884224D0022077
:102D000011902B201290039800280CDA4042039077
:102D10002D20129007E00A210398FDF7EBF93031DE
:102D20007F1E039039701199481E11900029F2DC22
:102D300003980028EFD1791E12980870307820216E
:102D400008404530BF1E387006A8C01BC01D039048
:102D500010980078002800D00120019941180298AD
:102D6000C0170918039809180498401A401E0490C7
:102D7000E00306D421461A9B199A049800F05EF8E5
:102D8000451910980078002803D01A9A199990478D
:102D90006D1CE00324D521461A9B199A049800F073
:102DA0004DF845191CE00098002807DB00990598AC
:102DB000884203DD1598405C199901E0199930208B
:102DC0001A9A904700986D1C401C00900298401E73
:102DD0000290002804D11A9A2E20199990476D1C50
:102DE0000199481E01900029DDDC05E038781A9A27
:102DF0007F1C199990476D1C0399481E0390002968
:102E0000F4DC21461A9B199A0498ACE62D000000C8
:102E10002B0000002000000000000000F8B5044670
:102E200000251E461746880404D405E039462020B4
:102E3000B0476D1C641EF9D52846F8BDFFB50446A1
:102E4000002581B01E46C80301D5302700E02027A9
:102E5000880404D505E038460399B0476D1C641E0C
:102E6000F9D5284605B0F0BD01B5044B01226946ED
:102E70000348FEF709FF009808BD0000FFFF0000AF
:102E8000FC000020FEF7D4F8FFF770F8FEF79EFF75
:102E9000FFF726F8FFF702F8FEF760FFFEF7D2FF14
:102EA0002748FDF7BFFE32212548FDF75BFE244889
:102EB000FDF746FD800538D52148FDF743FD214D3E
:102EC00080B22880FDF76CFA1F4E3146FDF76AF993
:102ED0000B21C943FDF7A3F9FDF778FA02460B462B
:102EE0001AA0FFF725FBA868FDF770FA00221C4B1B
:102EF000FDF7A2F907460C462888FDF751FA31463E
:102F0000FDF750F90B21C943FDF789F9FDF75EFA8A
:102F10003A462346FDF735FAFDF76CFAFDF756FA07
:102F200002460B460FA0FFF703FB06490422891C4B
:102F30001048FEF7FFFD1048FDF7C8FEB0E700009F
:102F4000180000200000002033335340766F6C746B
:102F5000616765203A2025312E3366560D0A000040
:102F60000000F83F4F5250203A2025312E3366564C
:102F70000D0A0000FC0000201027000000000000E7
:102F80000000000001020304060708090304060804
:102F90000C101820300000000001020304000000A3
:102FA000C02F00080000002018000000982500082D
:102FB000D82F00081800002068050000A825000888
:102FC0000000000000000000000000000000000001
:082FD0000000200000000000D9
:04000005080000C12E
:00000001FF
